:020000040000FA
:040000006E303A28FC
:040004000034003490
:08000800A000030EA100831209
:100010008B1C32288B1032181428B21C3228643002
:10002000010203183128182800001628172818285C
:1000300019281A281B281C281D281E281F283210A2
:10004000B214A810031005190314AA0DA90DA80DC8
:10005000B10B322832152A08AF002908AE00280853
:10006000AD00B21081010B11210E8300A00E200EF5
:02007000090085
:0C007400203084008001840A80300402E7
:10008000031C3C281230B100962183160C308505E4
:1000900087018312850187010730990000309A009B
:1000A000103083168E008312603083168F00831207
:1000B00000308316910000008312C830831681003F
:1000C000831231309000003083168C008312103080
:1000D0008B00B72181018E018F010B118B100B104A
:1000E0008C018B178220321998207821B40B80283C
:1000F000031085190314BA0DF0303A0203191A21BE
:10010000B82172286400321808000B1D08000B117A
:10011000B21032141230B100051D93283314831627
:10012000011383120800331083160117831208008D
:1001300032110130B7008B132030370783169B0034
:100140001C141A088312A400A500C030A5061030A4
:10015000370783169B001C141A088312A300003073
:10016000370783169B001C141A088312A2008B17F2
:10017000331CC02822090339A200A309A409A50938
:1001800022082D02031D142923082E02031D142901
:1001900024082F02031D142901303702031DD5281E
:1001A0003E18D5283E143F149E2102303702031D0D
:1001B000DE28BE18DE28BE143F14A121033037020A
:1001C000031DE7283E19E7283E153F14A4210430FB
:1001D0003702031DF028BE19F028BE153F14A721D1
:1001E00005303702031DF9283E1AF9283E163F1440
:1001F000AA2106303702031D0229BE1A0229BE16A3
:100200003F14AD2107303702031D0B293E1B0B297C
:100210003E173F14B02108303702031D1429BE1BBE
:100220001429BE173F14B321B70A09303702031847
:1002300008009B280130B600B400B500B700850166
:100240008701B213B6218220B40B39290310851916
:100250000314BA0DF0303A02031960295030B4008B
:10026000B51F8501B51F8701B50B39299630B5003B
:100270006C21321D23293211331C43292D090339E6
:10028000AD00AE09AF092F1CB2132F1C2329B21BDE
:1002900023292E182329B2178B1320303707BC00CF
:1002A0002F08BB00812110303707BC002E08BB008F
:1002B000812100303707BC002D08BB0081218B173E
:1002C00085018701B70AB6010130B5000930370250
:1002D000031C2329B72108003708B6080319B60004
:1002E000031908001130850013308700B603080099
:1002F0003F1C08003F101030BC003E08BB008121AD
:1003000008008B133B0883161C159A0083123C08C7
:1003100083169B0055309D00AA309D009C146400FC
:100320009C188F291C1183128B170800831610301C
:100330009B001C141A088312BE0008000130BE0086
:1003400008000230BE0008000430BE00080008307B
:10035000BE0008001030BE0008002030BE000800BB
:100360004030BE0008008030BE00080008000800D1
:100370008F08031908008F0107303E050319B02AC2
:1003800002303E05031D51105408EB3C03180512C2
:100390005118CD29D40BD829D229D4035408C83CEC
:1003A000031CD8290516F530D4005108013AD100B4
:1003B00002303E05031DD1105508E63C0318851296
:1003C000D118E529D50BF029EA29D5035508B93C00
:1003D000031CF0298516F030D5005108023AD100EF
:1003E00002303E05031D51115608DC3C0318051070
:1003F0005119FD29D60B082A022AD6035608B63C05
:10040000031C082A0514E630D6005108043AD1002E
:1004100002303E05031DD1115708F03C031885102A
:10042000D119152AD70B202A1A2AD7035708D73CE7
:10043000031C202A8514FA30D7005108083AD1004D
:1004400002303E05031D51125808E03C0318871086
:10045000511A2D2AD80B382A322AD8035808C13C01
:10046000031C382A8714EA30D8005108103AD1000A
:1004700006303E05031DD1125908D43C031807115C
:10048000D11A452AD90B502A4A2AD9035908A73C20
:10049000031C502A0715DE30D9005108203AD1003C
:1004A00006303E05031D51135A08BF3C03180710C0
:1004B000511B5D2ADA0B682A622ADA035A089C3C2F
:1004C000031C682A0714C930DA005108403AD100E9
:1004D00006303E05031DD1135B08D73C0318871275
:1004E000D11B752ADB0B802A7A2ADB035B08BE3C12
:1004F000031C802A8716E130DB005108803AD100C6
:1005000006303E05031D52105C08F13C031807122B
:1005100052188D2ADC0B982A922ADC035C08CF3C07
:10052000031C982A0716FB30DC005208013AD2005F
:1005300006303E05031DD2105D08E93C0318871103
:10054000D218A52ADD0BB02AAA2ADD035D08B23C29
:10055000031CB02A8715F330DD005208023AD2009E
:1005600018303E050319002BBE1DBC2A54083C3C24
:10057000031CBC2A85018701D40B0800D003463038
:10058000D4000B305002031DC62A05160A30500253
:10059000031DCB2A851609305002031DD02A0514ED
:1005A00008305002031DD52A851407305002031D60
:1005B000DA2A871406305002031DDF2A071505309A
:1005C0005002031DE42A071404305002031DE92AD7
:1005D000871603305002031DEE2A07160230500220
:1005E000031DF32A871501305002031DF72A12302C
:1005F0005002031C0800850187010C30D000080060
:1006000020303E0503194A2BD40B0B2B0508103A5A
:1006100085008230D400D50B122B0508203A8500C6
:100620007D30D500D60B192B0508013A85007330B3
:10063000D600D70B202B0508023A85008730D7005B
:10064000D80B272B0708023A87007730D800D90B40
:100650002E2B0708043A87006B30D900DA0B352BB4
:100660000708013A87005630DA00DB0B3C2B0708FD
:10067000203A87006E30DB00DC0B432B0708103A72
:1006800087008830DC00DD0B4A2B0708083A87001A
:100690008030DD0040303E050319C12B5408E63C94
:1006A00003180512D40B702B0516F030D40021303E
:1006B000DE0703186E2BB130D507FA30D607C830E5
:1006C000D7076430D8079630D907BE30DA07AA308A
:1006D000DB079A30DC07C430DD07702B8030BE00AA
:1006E0005508823C03188512D50B792B85168C3062
:1006F000D5005608653C03180510D60B822B05144F
:100700006F30D6005708913C03188510D70B8B2B00
:1007100085149B30D7005808D73C03188710D80B96
:10072000942B8714E130D8005908503C0318071166
:10073000D90B9D2B07155A30D9005A08873C03184E
:100740000710DA0BA62B07149130DA005B08BD3CCA
:1007500003188712DB0BAF2B8716C730DB005C0852
:10076000703C03180712DC0BB82B07167A30DC003C
:100770005D08A73C03188711DD0BC12B8715B1302D
:10078000DD0080303E050319C82B85018701DE019D
:0207900008005F
:084000000B00030007000100A2
:02400E00CC33B1
:10420000010003000300030003000200020002009B
:1042100002000000000000000000FF00FF00FF009F
:10422000000000000000000000000000000000008E
:104230000000C000C000C000C000FF00FF00FF0081
:104240000100C300F300CF00FF00C300F300CF0064
:10425000FF00C300F300CF00FF00FF00FF00FF00DE
:10426000FF00FF00FF00FF00FF00FF00FF00FF0056
:10427000FF00FF00FF00FF00FF00FF00FF00FF0046
:10428000FF00FF00FF00FF00FF00FF00FF00FF0036
:10429000FF00FF00FF00FF00FF00FF00FF00FF0026
:1042A000FF00FF00FF00FF00FF00FF00FF00FF0016
:1042B000FF00FF00FF00FF00FF00FF00FF00FF0006
:1042C000FF00FF00FF00FF00FF00FF00FF00FF00F6
:1042D000FF00FF00FF00FF00FF00FF00FF00FF00E6
:1042E000FF00FF00FF00FF00FF00FF00FF00FF00D6
:1042F000FF00FF00FF00FF00FF00FF00FF00AA001B
:00000001FF
